:020000040000FA
:100000000030860085000728AD0A0B110900031394
:10001000831207309F00A0308B008316C53081000B
:100020000030860004308500831220308400800177
:10003000840A041F17280030AB0019222130E42362
:10004000AE002430E423B1002230E423B800B30032
:100050000230E423BE001E30E423C0002330E4233A
:10006000AC00AC182C150430B5001930C3003C129C
:100070000510E9213F205A20F92027223A28203074
:10008000B9001330A900043005052A0603194D28CC
:10009000B90B50280430AA063F282A30A900482866
:1000A000043005052A0603194128BF20DB20A90BCF
:1000B000502808002508A1002608A2002708A30050
:1000C0002808A400A501A601A701A80125308400E5
:1000D0006C2074207C2008000830A9009D20A020FE
:1000E000800DA90B6E280800840A9D20A020800D99
:1000F0009D20A020800D0800840A0430A9009D20C6
:10010000A020800C840A9D20A020800CA903031944
:100110008B2884037F28800E8403800E080004301F
:1001200005052A060319B90A08002A1D9A28051D83
:100130009728080005199A2808002A199A2897284C
:10014000AD01BF20043005052A060319AA28AD1801
:10015000B828A128BF20BF20BF20B9018F20BF2011
:10016000BF208F20BF20DB208F2002303902080003
:100170002030C2002F08C100CE2395201E282B1846
:10018000CE288611010C7F390319CA282F02031CBF
:1001900006110800AF08031D061508000611010C22
:1001A0007F390319D7282F02031C86110800AF08D6
:1001B000031D86150800BC1CF62832082F02031CFC
:1001C000F42803103B0D2C1C3B08323E2C180A3E31
:1001D000A000010CA002031808007D3C031CF228BB
:1001E00005100800051408000514BF28AC180510F8
:1001F000BF2821082502031D202922082602031DED
:10020000202923082702031D202924082802031D72
:1002100020292108031D1029013023020319742A03
:1002200021082E0203191A292C1F20292108310226
:10023000031D2029BF20230824020319AD292129E9
:1002400008003C162808FE3E03194829FF3E031902
:100250000613FF3E03198613FF3E03194E29FF3E86
:1002600003199921FF3E03197E21FD3E03195329ED
:10027000FF3E03190617FF3E03198617FF3E0319B9
:100280004B29FF3E0319A321FF3E03198C21C729E7
:100290002308073C72292308F83E72292308073CEB
:1002A00003186629722908302702031C72290319D2
:1002B0002029FD3E03190617FF3E03198617FE3E4F
:1002C0000319A321FF3E03198C21C72903197E219D
:1002D000FF3E03199921FE3E03198613FF3E0319C1
:1002E0000613C729240801392B060319C729240836
:1002F0000139AB0021220130A300C729AC1E8A2995
:10030000BC1E0800B9002230E423B800B300BC12C0
:100310003908080085100800AC1E9729BC1A08008F
:10032000B9000130B800B300BC16390808008514C4
:1003300008002C1DA129AC1C9F29BC1008003C11F1
:100340000800051008002C1DAB29AC1CA929BC1401
:1003500008003C15080005140800BF202308013AD6
:10036000031DC2293C18B829FF30B4000430B50081
:100370003C186B223C18C7293C14AB090130AB0573
:100380002122C729AC18BC143C1CC7293C10BF2033
:10039000E9212308013A0319E6292308BB003C1987
:1003A000DE290310BB0DAC1FE229A2080319E229C4
:1003B000221CBB0AA218E229BB0AE2293C1EE22940
:1003C0003030BB073B08E423B2000800B201AF01A4
:1003D00008002C1A0B2A2B18FC2906128616AF08C7
:1003E00003198612AC1D86163C1A0800A218FA29B9
:1003F000061308000617080086120616AF08031930
:100400000612AC1D06163C1A0800A218092A86130B
:100410000800861708002B18132A0612A218861641
:10042000A21C861208008612A2180616A21C06122A
:1004300008002030E423AF00B2002530E423AB00F5
:1004400008002530C2002B08C100CE230800380860
:10045000013C031D2E2A3208AF0008003C1232086E
:100460002F0203190800B30B08003E082F020318DF
:10047000422AB20803193F2A3E08AF00422AAF01C0
:10048000B30A080032082F02031C482AAF03492A86
:10049000AF0A3808B300AD012630E4232F08BF00AF
:1004A000C10B532A572ABF070318AD0A502A04303C
:1004B000C100AD0CBF0CAD13C10B592AAD08031818
:1004C000632AAD0CBF0C2730E4233F084102031C14
:1004D0000030B3070800B40B08006F2A0800FF3093
:1004E000B400B50B0800A82AC30B0800C22BB60045
:1004F000B60A0B30BC1BEA2BB60B7F2A0800861607
:100500000616EA2386120612EA237C2A0230B60077
:100510002F307A2A95222308013A03198A2A952234
:100520002308013A031D8F2A08003F205A20210882
:100530002502031D952A22082602031D952A230859
:100540002702031D952A24082802031D952A080066
:10055000BC1009307722013077228A22F023B903B8
:100560000319D92AB9030319E12AB9030319EC2A9B
:10057000B9030319262BB90303193C2BB90303193B
:100580004E2BB9030319562BB9030319682BB90372
:1005900003197B2BB90303198D2BB9030319A02B66
:1005A0000430B9020319AE2B21080319BA2B862295
:1005B000AD2A77228A222130C2002108C100CE2331
:1005C000AB2A77228A222230C200F0233908C100E8
:1005D0002230C200CE23AB2A77228A22F023C20027
:1005E0000310C20D210803190B2B10303902031C14
:1005F000FB2A8622ED2A390877228A22F02303106B
:10060000B90DB91F052B8622FD2A3908C100CE235A
:1006100001307722ED2A0630B600E423B900B60394
:100620003603E423B9020310390CC1073608C200AF
:10063000CE2383169C181A2B8312B60A1E3036025C
:100640000318AB2AB60AB60A36080D2B77228A227F
:10065000F02304303902031C2F2B8622272B233052
:10066000E423E730C105B9033918C115B91841169B
:100670002330C200CE23AB2A77228A22F023033014
:100680003902031C452B86223D2B2330E423C11263
:10069000391CC1162330C200CE23AB2A77228A220E
:1006A0002430C2002108C100CE23AB2A77228A223F
:1006B000F02303303902031C5F2B8622572B233093
:1006C000E4234113391C41172330C200CE23AB2A47
:1006D00077228A22F02305303902031C712B8622EF
:1006E000692B2330E423F830C1053908C1042330D5
:1006F000C200CE23AB2A77228A22F02303303902AC
:10070000031C842B86227C2B2330E423C113391C49
:10071000C1172330C200CE23AB2A77228A22F023CE
:1007200004303902031C982B21303902031C9A2B08
:1007300086228E2B2630C2003908C100CE23AB2A78
:1007400077228A22F023B908031DA82B8622A12B29
:100750002730C2003908C100CE23AB2A8A22F023F9
:1007600003303902031CB62B8622AE2BBC13391C76
:10077000BC17AB2AFF30B4000430B500013077223B
:1007800091211E288A228A222130C2002108C1001C
:10079000CE231930C300093077221E284108831662
:1007A0009A008312420883169B008B131C129C1123
:1007B0001C1555309D00AA309D009C141C119C18DE
:1007C000DF2B83128B17080083169B001C141A085A
:1007D00083120800AD01AD02AD08031DEC2B08002B
:1007E000B901A11FF62BB90A211FB90AA11EFC2BC2
:1007F0000330B907211EB907A11D022C0930B90722
:10080000211DB907A11C082C1B30B907211CB907F1
:04081000390808009B
:02400E00703F01
:104200000000000012000000140015001600180045
:104210001A001C001E0020002200250028002B0090
:104220002E00320036003A003E00430048004E00A7
:1042300054005A00600067006E0075007C000000AA
:1042400000002A000400A0002A00000010001E0048
:10425000000000000000000000000000000000005E
:104260000000000008000A000C000E001000120000
:10427000150018001B001E002100250029002D003C
:10428000FF00FF00FF00FF00FF00FF00FF00FF0036
:10429000FF00FF00FF00FF00FF00FF00FF00FF0026
:1042A000FF00FF00FF00FF00FF00FF00FF00FF0016
:1042B000FF00FF00FF00FF00FF00FF00FF00FF0006
:1042C000FF00FF00FF00FF00FF00FF00FF00FF00F6
:1042D000FF00FF00FF00FF00FF00FF00FF00FF00E6
:1042E000FF00FF00FF00FF00FF00FF00FF00FF00D6
:1042F000FF00FF00FF00FF00FF00FF00FF00FF00C6
:00000001FF
